:020000040000FA
:100000008B018A018301A828F000030E8301F1000F
:100010000408F3008C1E5428981C18195128181C29
:1000200028284611C5011A08C000C6196B28603A75
:10003000031925284008410603194828A03A031946
:100040002528603A03193E286B28C40146156B2801
:100050002030450784001A08461D6B288000C4061E
:10006000C50A2030840000080F39023E4506031DF2
:100070006B28461144080319C6156B280614203056
:1000800099008316981C4228831220309900622818
:10009000461C6B28061483160C168312C201C61464
:1000A00058281A08181218160C1E6B28C61C62282D
:1000B000A0304207840000089900C20AC30B6B28D5
:1000C0004610C6108316981C63280C1267286828EF
:1000D00069288312061073088400710E8300F00EE5
:1000E000700E090082073F3406345B344F346634A7
:1000F0006D347D3407347F346F34CF19DF01DF086E
:10010000031908000301DF1A01305F1B0230DF18FA
:100110000330DF01610782078A2AD12A9F2AE42A55
:10012000A82A912A9A2AE42AD42AB42AD92AE42A83
:100130000800FE2A0A2BA828FE2AE92AF62AA8285F
:10014000FE2A132B1D2BA828B72AA42AA22AE42AA8
:100150009801193085008601831606308600263006
:10016000850020308C00813081000B308E00003003
:100170009F00831205309F003130900020308400B2
:100180008001840A841FC0285C1421226623242352
:10019000C0308B004030DA00DB00FF30E200851A0F
:1001A000052901307923D300D4016030D500C9215D
:1001B0008E018F010C10FA200C18FF204618DB2846
:1001C000CE21013090008E018F010C10D422E0214D
:1001D00035161030BB00FA200C1CEB280C10BB0BA2
:1001E000EB28FA200C1831237D20F1288C1C080004
:1001F0008C100800F6203122C6190E2108000C10C0
:100200007930DA000730DB0008000023013090006D
:10021000C91A5E23F62031227D2008292008613A80
:10022000031D3E292108031D2029CF18C729CF11FE
:10023000CF144F107930DA003F30DB007C22C42924
:10024000013A031D3029CF11CF104F1053086E22F1
:100250007C224F080B390319C429C611E021C42997
:10026000033A031DC729CF19C729CF15CF104F1047
:100270006D30DA007330DB007C22C429033A031DA1
:100280004E292108223A031DC7292208CF00CF1981
:100290003829CF181A294F1866292629013A031D33
:1002A0005A292108213A031DC7292208C70023081B
:1002B000C800C7292008813A031D6C292108031DA5
:1002C000C7294F18C729CF11CF104F147930DA0042
:1002D0006D30DB007C22C4292008E13A031D7B2914
:1002E0002108883A031DC7296D30DA004030DB0051
:1002F000CC30E200C729033A031D88292108F039D0
:10030000203A031DC72949155308D200D501A82951
:10031000013A031D9B292108403A031DC7292208E1
:100320003F39031DC72923085306031DC729491454
:100330007C223516C729073A031DB8292108F03950
:10034000031DC72949115308D20023081F39D500BE
:10035000A21BD516211CA11855172119D517220843
:100360007F39D4004910A11949147C223516C729B8
:10037000013A031DC7292108F039103A031DC72986
:1003800049152508D200A5290030E1007C22C611BC
:10039000080021300C22213014221D2A21300C2289
:1003A000243014221D2A80300C221D2A21300C22D8
:1003B000803014221D2A21300C22813014221D2A63
:1003C000E3300C220030142200301422530814228F
:1003D0001D2AE4300C221030551B1230D51B13306F
:1003E000142200301422530814225408D51A8038DD
:1003F000142249107C225308FB0001307F231D2A60
:10040000E4300C222030142200301422530814222D
:1004100055081F391422F929BC00C6190E214618A7
:100420000D2AC201C3013C08BD00A030430784006F
:100430003D088000C206C30A080042081422461480
:100440000800003079231F394038C100BD003D0E3F
:10045000BD063D0CBD063D19BD0A3D0C0318C11774
:1004600008000B1D08000B115C08851ADD0418300C
:1004700085000310DC0DDC1B5C145D22E21F08000C
:100480005B085C05031D05125A085C05031D8511F8
:100490005C1C08005E095D05DF000319512A473026
:1004A000E0005D08DE00DD015E0803190800E00BD6
:1004B0000800DF001C30E00008003E3085050F30EA
:1004C00086055C180514DC1A85175C1B05175C0D86
:1004D0008400840D040DF03986040800DB00DA0185
:1004E0000A30DA0ADB020318712A5B077220DB008C
:1004F0005A037220DA000800FF30E108031DDF30E4
:100500004918CC30CF18C3304F18C330CF19C3307F
:10051000E20008003830DA00DB010430E1007C2220
:100520000800D30A6430530601300319D300E021D8
:1005300053086E2AD30363300319D300972A10306F
:10054000D506002A0230A62A0130A62AD5060022A6
:100550000830D5180130DB00083055180130DA00BA
:100560001830E1007C2208002030D506E921590826
:10057000031DD42AD51EC52A5E30DA000830551B6B
:100580004030D51B0130DB00CD2A0830551B4030F0
:10059000D51B0130DA005E30DB000830E1007C2240
:1005A00008002030D506E9210030E1007C22530804
:1005B0006E2A5908031D08008030D51F4030551B96
:1005C000C030D506E921B72A4F18DB29CF18E52A14
:1005D000D62900307923FB00FB0A20307B0601304E
:1005E0000319FB0000307F237B086E2A003079233B
:1005F000FB00FB031F300319FB00F22AC91D032B6C
:10060000C9117730052BC9157330DA00DB010C30C6
:10061000E10008001430C91D1030E100C9190800BC
:10062000003079236E2A02307923FB00FB0A7B1A03
:10063000FB037B08D80002307F2B02307923FB00BC
:10064000FB03FB1BFB01192B831606309200831260
:100650007C309200023079230F39D8000C3097009B
:1006600008000C100310E21B0314E20D46180800EA
:10067000380C1F39BD005906031908003D08D90080
:10068000351A5C2B551B4D2BD51B572B3D0C0F39A9
:10069000013A031D013AD400E92904303D02031C4C
:1006A000BD013D0C031810381F39D400E929BD0DD8
:1006B0003D0D7C39D400E929351208000C10C9120F
:1006C0006108143A031D080038086E2A0610C60196
:1006D000C501831603309900643098008312D0302E
:1006E00098000301FF3E031D722B1A081A081A080E
:1006F000080083169B001C141A0883120800792333
:100700007B06031908007B0883169A001C158B13BF
:1007100055309D00AA309D009C148B171C119C180D
:060720008F2B831208007C
:02400E00503F21
:06420000010003000000B4
:10422000533469346D3470346C34653420344D3417
:10423000613475347334203476342E3433340A3494
:1042400046342E3443346134C334B134613464347D
:1042500061342D343E3448342E344834613466346D
:1042600074346D3461346E346E340A34313439341C
:0C4270002F34303431342F3433343034E8
:00000001FF
